:100000000C9417060C9429290C9456290C943F063D
:100010000C943F060C943F060C943F060C943F064C
:100020000C943F060C943F060C940D0C0C943F0668
:100030000C943F060C943F060C943F060C943F062C
:100040000C9483290C943F060C943D2D0C94782D30
:100050000C943F060C943F060C943F060C943F060C
:100060000C943F060C943F067D1C841C841C7D1C54
:10007000841C841C841C841C841C841C841C841C80
:10008000841C841C841C841C841CF21B841C841C03
:10009000841C841C841C551B841C841C841C841C90
:1000A000841C841C841C841C841C841C841C841C50
:1000B000841C841C841CFE1BFE1BFE1BFE1BFE1BE3
:1000C000FE1BFE1BFE1BFE1B841C841C841C841C4C
:1000D000841C841C5A1BFD1BFD1BFD1BFD1B841C6B
:1000E0000E1C161C1E1C261C2E1C361C3E1C461CE0
:1000F000501C5A1C641C6E1CA11B611B841C841C9C
:10010000841C841CF21B841C841C841C841C841C82
:10011000841C841C841CFC1BFC1BFC1BFC1B841C03
:100120000E1C161C1E1C261C2E1C361C3E1C461C9F
:10013000501C5A1C641C6E1CA11B611B841C841C5B
:10014000841C841CF21BB51CB51CB51CB51CB51C4D
:10015000B51CB51CB51CB51CB51CB51CB51CB51C17
:10016000D51DD51DD51DD51DD51DD51DFC1C061DA8
:10017000101D1A1D801D8A1D981DA91D461EB61E24
:10018000871E8C1E911E961E9B1EA01EA51EB61EAF
:10019000B01EBD25D225DE25E725F4251A26222608
:1001A00045263226456E746572206D656E752E2E5D
:1001B0002E00546F67676C6564206D6963726F50C1
:1001C000504D00546F67676C656420696E76657288
:1001D0007465642050504D2100546F67676C6564EE
:1001E000205458206D7574696E672100546F6767DD
:1001F0006C65642074656C656D657472792100505E
:10020000726F746F636F6C206572726F72207769A2
:1002100074682052580054696D656F757420776852
:10022000656E20636F6E6E656374696E6720746FB0
:1002300020525800507265737320616E79206B658F
:100240007920746F2063616E63656C00436F6E6E1E
:10025000656374696E6720746F2052582C20706F2C
:100260007765722075702074686520525820287751
:100270006974682062696E6420706C7567206966B5
:10028000206E6F74207573696E6720616C77617979
:10029000732062696E642900546F67676C6564201F
:1002A00027696D6D656469617465206F757470751B
:1002B000742700546F67676C65642027736C6176E0
:1002C00065206D6F64652700546F67676C656420F7
:1002D00027616C776179732062696E642700546FBF
:1002E00067676C65642050504D206368616E6E6571
:1002F0006C206C696D6974005365742052535349C6
:1003000020696E6A656374696F6E206368616E6EE2
:10031000656C2028303D3D64697361626C6529001D
:100320005365742050504D206D696E696D756D2058
:1003300073796E630053657420626561636F6E202C
:10034000696E74657276616C0053657420626561D4
:10035000636F6E2064656C6179005365742062651B
:1003600061636F6E206672657175656E6379206971
:100370006E20487A3A20303D64697361626C652C66
:100380002050783D504D52206368616E6E656C2040
:10039000782C2046783D465253206368616E6E6526
:1003A0006C2078005365742050574D2073746F7023
:1003B0002064656C61792028302064697361626C07
:1003C00065642C20312D323535203D3D20302E31D5
:1003D00073202D2035306D696E29005365742050CF
:1003E000504D2073746F702064656C6179202830E3
:1003F0002064697361626C65642C20312D3235355F
:10040000203D3D20302E3173202D2035306D696E1A
:100410002900536574206661696C736166652064A8
:10042000656C61792028302064697361626C656451
:100430002C20312D323535203D3D20302E3173209A
:100440002D2035306D696E29002A2A2A2A2A2A2A67
:100450002A2A2A2A2A2A2A2A2A2A2A2A2A2A2A2AFC
:100460002A2A2A2A2A2A0052582041636B656420CE
:100470002D2072657665727420737563636573737E
:1004800066756C21002A2A2A2A2A2A2A2A2A2A2A36
:100490002A2A2A2A2A2A2A2A2A2A2A2A2A2A2A2ABC
:1004A0002A2A002A2A2A2A2A2A2A2A2A2A2A2A2AD6
:1004B0002A2A2A2A2A2A2A2A2A2A2A2A2A2A2A2A9C
:1004C0000052582041636B6564202D207570646173
:1004D0007465207375636365737366756C21002A98
:1004E0002A2A2A2A2A2A2A2A2A2A2A2A2A2A2A2A6C
:1004F0002A2A2A2A2A2A2A2A2A2A2A2A0056616CE1
:1005000069642063686F69636573206172653A206E
:100510005B315D2D5B31365D20286368616E6E65F1
:100520006C20312D31362900536574206F7574703D
:10053000757420666F7220706F727420005B585D56
:100540002061626F7274206368616E6765732061F9
:100550006E64206578697420525820636F6E6669F6
:1005600067005B535D207361766520736574746901
:100570006E677320746F205258005B525D20726565
:10058000766572742052582073657474696E67734F
:1005900020746F2064656661756C747300557365B3
:1005A000206E756D62657273205B312D445D207421
:1005B0006F206564697420706F727473205B452DC1
:1005C000515D20666F722073657474696E67730085
:1005D000202D20726563656976657220636F6E6693
:1005E0006967757261746F722C207278207377203E
:1005F000000A0A6F70656E4C52536E672000536597
:10060000742073657269616C2062617564726174D3
:10061000653A200056616C69642063686F696365A0
:10062000733A2031202D20342B34202F2032202DDE
:100630002038202F2033202D20382B34202F203419
:10064000202D203132202F2035202D2031322B3407
:10065000202F2036202D203136005365742043682A
:10066000616E6E656C20636F6E6669673A20005339
:1006700065742044617461726174652028302D3284
:10068000293A200053657420486F70206368616EBA
:100690006E656C7320286D61782032342C20736570
:1006A0007061726174656420627920636F6D6D6141
:1006B00073292076616C69642076616C756573209E
:1006C000312D3235353A2000536574206368616EF0
:1006D0006E656C2073706163696E672028783130B5
:1006E0006B487A293A200053657420524620706F77
:1006F0007765722028302D37293A20005365742001
:100700005246206D616769632028686578292065F5
:100710002E672E20307844454144463030443A20FC
:10072000005365742062617365206672657175653A
:100730006E63792028696E20487A293A20005B5A36
:100740005D20656E74657220726563656976657299
:1007500020636F6E66696775726174696F6E20756C
:1007600074696C79005B465D20646973706C6179B3
:100770002061637475616C206672657175656E6366
:100780006965732075736564005B525D2063616CFD
:1007900063756C6174652072616E646F6D206B654A
:1007A0007920616E6420686F70206C697374005BDF
:1007B000495D207265696E697469616C697A65204A
:1007C00073657474696E677320746F20736B6574DE
:1007D00063682064656661756C7473005B585D20A6
:1007E000726576657274206368616E6765732061F7
:1007F0006E642065786974206D656E75005B535D6D
:1008000020736176652073657474696E67732074F4
:100810006F20454550524F4D20616E6420657869C8
:1008200074206D656E7500557365206E756D62651B
:100830007273205B302D395D20746F20656469749C
:1008400020706172616D657465727300202D205394
:10085000797374656D20636F6E6669677572617414
:10086000696F6E000A0A6F70656E4C52536E672096
:10087000005129204F7574707574206265666F721F
:1008800065206C696E6B20283D465329203A200074
:10089000502920536C617665206D6F646520286552
:1008A00078706572696D656E74616C293A20004FCD
:1008B000292054696D65642042494E4420617420AA
:1008C0007374617274757020203A20004E29205094
:1008D000504D206F7574707574206C696D69746506
:1008E0006420202020203A200044495341424C45B6
:1008F00044004D292050504D205253534920746FCD
:10090000206368616E6E656C202020203A20004CC8
:10091000292050504D206D696E696D756D20737979
:100920006E63202875732920203A200044495341E2
:10093000424C4544004B29204661696C73616665F1
:1009400020626561636F6E20696E74762E20283197
:100950002D32353573293A20004A29204661696CC9
:100960007361666520626561636F6E2064656C61AA
:10097000792028302D323535203D3E20313073200E
:100980002D203135306D696E293A200049292046E5
:1009900061696C7361666520626561636F6E206674
:1009A00072712E203A200048292050574D20737430
:1009B0006F702064656C6179202020202020203A0F
:1009C000200047292050504D2073746F70206465BB
:1009D0006C6179202020202020203A200046292008
:1009E0004661696C736166652064656C617920207D
:1009F00020202020203A200050574D206368616E4F
:100A00006E656C200066756E6374696F6E3A2000C7
:100A10002920706F72742000506F776572546F7761
:100A2000657200445446205548462033322D626991
:100A3000742031306368004F70656E4C52536E679E
:100A40005258206D696E6920342F36636800466CF9
:100A50007974726F6E2F4F72616E676552582055B0
:100A600048462038636800525820747970653A20EF
:100A70000044697361626C656400487A00203D3D02
:100A8000200043616C63756C617465642070616300
:100A90006B657420696E74657276616C3A200042F1
:100AA00029204D6963726F202868616C6629205087
:100AB000504D202020203A00412920496E76657251
:100AC0007465642050504D20696E20202020203A0B
:100AD000003029204D7574652062757A7A65722020
:100AE000286D6F73746C79293A0039292053657227
:100AF00069616C2062617564726174653A00736D3E
:100B0000617274506F7274004672536B7900547244
:100B1000616E73706172656E740044697361626CBA
:100B200065640038292054656C656D657472793A86
:100B300020202020202020003729204368616E6E6D
:100B4000656C20636F6E6669673A20200036292045
:100B500044617461726174652028302D32293A2015
:100B6000202000352920486F70206368616E6E6513
:100B70006C733A2020202020003429204368616EC5
:100B80006E656C2073706163696E673A2020003374
:100B90002920524620706F7765722028302D372922
:100BA0003A202020003229205246206D6167696377
:100BB0003A202020202020202020003129204261BE
:100BC0007365206672657175656E63793A202020C1
:100BD0000000000000240027002A0000000000257B
:100BE0000028002B0000000000230026002900043C
:100BF00004040404040404020202020202030303C4
:100C000003030301020408102040800102040810BD
:100C1000200102040810200000000700020100006B
:100C2000030406000000000000000000202F112433
:100C30001FBECFEFD8E0DEBFCDBF13E0A0E0B1E034
:100C4000E2E8F0E602C005900D92A839B107D9F7A5
:100C500016E0A8E9B3E001C01D92AB35B107E1F79A
:100C60001CE0CEE2DCE004C02297FE010E941C30B2
:100C7000CC32D107C9F70E94652F0C943F300C94F9
:100C80000000A0E0B0E0E7E4F6E00C94EB2FEC010C
:100C9000A880B980CA80DB80A114B104C104D1044A
:100CA00041F484E2A82E89EDB82E8BE5C82E87E0AA
:100CB000D82EC601B5012DE133EF41E050E00E948E
:100CC000C82F27EA31E440E050E00E94742F7B01F6
:100CD0008C01C601B5012DE133EF41E050E00E94E7
:100CE000C82FCA01B9012CEE34EF4FEF5FEF0E941D
:100CF000742F6E0D7F1D801F911F97FF04C06150E0
:100D0000704080409048688379838A839B839B01ED
:100D1000AC015F77B901CA01CDB7DEB7EAE00C9448
:100D200007300E944106089581EB92E00E9441063F
:100D300008956093B1027093B2028093B3029093CE
:100D4000B4020895A0E0B0E0E8EAF6E00C94E42FE5
:100D5000EC012B016A016115710519F0FB0191830A
:100D60008083C114D10449F0C6010297839728F00B
:100D700020E030E040E050E0DCC0A9908A2D90E017
:100D80000E943430892BC9F7FDE2AF1621F4A990F7
:100D90003324339405C08BE2A81609F4A9903324B8
:100DA000C114D10421F0E0E1CE16D10411F5F0E335
:100DB000AF1669F48881883711F0883541F4A9802D
:100DC000229682E0382A20E1C22ED12C12C0C11412
:100DD000D10479F4E0E3AE1659F199E9E92E99E9E5
:100DE000F92E99E9092F99E1192F8AE0C82ED12C03
:100DF0003AC0FAE0CF16D10491F080E1C816D104D0
:100E000029F0E8E0CE16D104F9F415C0BFEFEB2EBF
:100E1000BFEFFB2EBFEF0B2FBFE01B2F24C0A9E9B4
:100E2000EA2EA9E9FA2EA9E90A2FA9E11A2F1BC077
:100E3000F8E0CF2ED12CEFEFEE2EEFEFFE2EEFEFFE
:100E40000E2FEFE11E2F0FC09601442737FD40956E
:100E5000542F6FEF7FEF8FEF9FEF0E94A62FC901F6
:100E6000DA017C018D0120E030E040E050E060E0FC
:100E70003601882477FC8094982C70EDB72EBA0C3C
:100E8000F9E0FB1570F48A2D81548A3118F499EC3D
:100E9000B92E06C08A2D81568A3148F589EAB82EC6
:100EA000BA0C8B2D90E08C159D050CF56F3FE9F089
:100EB000E216F30604071507B8F0CA01B901A40148
:100EC00093010E94742F9B01AC018B2D90E0A0E058
:100ED000B0E0280F391F4A1F5B1F281739074A0740
:100EE0005B0710F061E001C06FEFA990C6CF41141D
:100EF000510451F0662311F0219703C031FE04C064
:100F00002297F201D183C08330FE07C050954095EF
:100F1000309521953F4F4F4F5F4F67FF0AC082E2E8
:100F200090E090935A06809359062FEF3FEF4FEFD2
:100F30005FEFB901CA01CDB7DEB7E1E10C94003033
:100F4000FC0188279927E89421912032E9F3293080
:100F500010F02E30C8F32B3241F02D3239F4689462
:100F600004C00E94F507820F911D219120532A3061
:100F7000C0F31EF4909581959F4F089548E953E082
:100F80000E94C3070895009731F4DA018D919C9176
:100F9000009709F40EC0DC01FB013D912191222351
:100FA00019F03217C9F3FACF332331F4DA011D9265
:100FB0001C928827992708951197AF93BF93FB013F
:100FC0003D912191321771F4332321F48827992719
:100FD000119702C01E921196FA01A193B0839F91BE
:100FE0008F910895222369F7EACF7AE0979F902D99
:100FF000879F802D910D1124089580919A0381304F
:1010000019F482E080939A0380919A03833019F453
:1010100084E080939A030895009721F19C0140E0B9
:1010200050E068E478EE81E090E00E94C82FC901AA
:10103000DA018F3F9105A105B10531F028F08FEF5E
:1010400090E0A0E0B0E008C00097A105B10521F450
:1010500081E090E0A0E0B0E08093B3008091B00028
:10106000806103C08091B0008F7E8093B0000895AE
:10107000E3E0F0E089E080935700849190E086708F
:10108000863009F491E0892F08951F93182F0E944C
:101090003808882379F09FB781E08093A105F89400
:1010A000A89588E18093600010936000112309F0F7
:1010B000A8959FBF1F910895382F20E08091330598
:1010C000909134058227932740E061E270E19C0112
:1010D000220F331F97FF04C0C9018627972701C03D
:1010E000C9014F5F483099F79093340580933305D9
:1010F000089587E38093D00380E092ECA1E0B0E014
:101100008093D1039093D203A093D303B093D403DD
:1011100087E08093DD0380EC9AECA9E8B6E3809346
:10112000D5039093D603A093D703B093D80385E05B
:101130008093DE038DEE9EEFADEABEED8093D90382
:101140009093DA03A093DB03B093DC03AFEDB3E03D
:1011500080E090E0863010F0E0E004C0FC01EF5742
:10116000FC4FE081ED9301968831910599F782E07B
:101170008093F7038AE08093F803089580EC97EF5B
:10118000AAEBB7E380939D0390939E03A0939F03E4
:10119000B093A00380E090E0A0E0B0E58093A103CD
:1011A0009093A203A093A303B093A403E5EAF3E012
:1011B00080E081938F5F8031E1F708958436910557
:1011C00020F4BC0180E090E025C08E3B910550F4F6
:1011D0008A559040BC0180E090E02AE030E040E099
:1011E00050E016C0823D910550F4845B9040BC01F4
:1011F00080E090E024E630E040E050E009C08D5C03
:101200009040BC0180E090E028E532E040E050E012
:101210000E94742F24E630E040E050E00E94742FDA
:10122000089590E08C599F4F0E94DE080895DC01DC
:101230009896EC91F0E0E770F070E758FC4F8081F1
:1012400008958F929F92AF92BF92CF92DF92EF92CA
:10125000FF920F931F938C010E941709D801979654
:101260002C9130E043E150E0249FF001259FF00DE8
:10127000349FF00D1124EB54FD4F80809180A280AB
:10128000B38090E00F96AA2797FDA095BA2FBC01D6
:10129000CD0120E43FE14DE750E00E94742FA5010D
:1012A00094010E94A62F69017A0180ED97E0A0E0E9
:1012B000B0E0C80ED91EEA1EFB1ED80198968C918C
:1012C000887181F060E07EEE8AEB9BE0A5019401DD
:1012D0000E94A62F28513C4F4F4F5F4FC20ED31E86
:1012E000E41EF51E87EE93E0A0E0B0E0C80ED91E24
:1012F000EA1EFB1EC701B60128EE33E040E050E0D5
:101300000E94A62FCA01B90128EE33E040E050E068
:101310000E94742F1F910F91FF90EF90DF90CF905C
:10132000BF90AF909F908F9008958F3F910509F0E7
:1013300010F480E0089522E08030920710F481E0FC
:1013400008958050934010F083E0089582E008955E
:10135000CF92DF92FF920F931F93CF93DF93F82FDB
:10136000EB016A01182F1695E0E088819981D6017A
:101370008C938A819B8111968C9311978C819D818E
:1013800012968C9312978E819F8113968C9313974C
:10139000288139814A815B816C817D818E819F8129
:1013A0009295990F990F907C832F8370982B852F9E
:1013B0008370880F880F982B872F83708295807F8A
:1013C000982B14969C9385E090E0C80ED91E289621
:1013D000EF5F1E1750F6F0FF21C0888199810E94AF
:1013E0009509F82E8A819B810E949509182F8C817E
:1013F0009D810E949509082F8E819F810E949509E9
:10140000F294FF0CFF0C70ECF7221295107F1F294D
:10141000182B000F000F012BD6010C93DF91CF91F9
:101420001F910F91FF90DF90CF90089523E08032BD
:10143000920718F420E030E026C023E0883E9207AF
:1014400048F49C012F51334054E0369527955A9526
:10145000E1F719C027E0803D920720F49C012C5D44
:10146000334011C028E08839920718F02FEF33E09D
:101470000AC09C01285C374044E0369527954A9580
:10148000E1F72D503C4FC90108958C30910548F487
:101490009C0174E0220F331F7A95E1F7285D3C4FE1
:1014A00017C023E0843F920720F49C0124523C4F54
:1014B0000FC024E08030920718F020E938E008C01F
:1014C0009C012657334F64E0220F331F6A95E1F7E2
:1014D000C90108959C013695279525753575821BA0
:1014E000930B9C0136952795369527952373337377
:1014F00083739373280F391FC901E4E0969587958C
:10150000EA95E1F7820F931F8F709F7021E031E021
:10151000AC01429FC001439F900D529F900D11243A
:10152000892F0895882339F02D9800002B9A000008
:101530002D9A000008952D9800002B9800002D9AF8
:10154000000008952D9A000083B12D98000090E0CE
:10155000B4E096958795BA95E1F7817008950F9359
:101560001F93082F5C9A2D985C9810E0802F80784C
:101570000E94920A000F1F5F1830C1F72D981F912B
:101580000F9108958F770E94AF0A08950F931F93CC
:10159000082F10E0802F80780E94920A000F1F5FB2
:1015A0001830C1F72D981F910F9108950F931F9335
:1015B0002D9880E000E0182F110F0E94A20A810FE1
:1015C0000F5F0830C1F71F910F9108950E94C20A62
:1015D0000E94D60A5C9A08951F93162F80680E9475
:1015E000AF0A812F0E94C60A5C9A1F9108951F932B
:1015F0001091D9031827E0EDF3E0E80FF11D89E71A
:1016000067850E94EC0A8DE3612F0E94EC0A82E458
:10161000612F0E94EC0A1F91089586E20E94E60A5B
:1016200008950F931F938C018CE1F80164810E944F
:10163000EC0A8DE1F80165810E94EC0A8EE1F80167
:1016400066810E94EC0A80E2F80167810E94EC0A40
:1016500081E2F80160850E94EC0A82E2F80161856E
:101660000E94EC0A83E2F80162850E94EC0A84E29F
:10167000F80163850E94EC0A85E2F80164850E9406
:10168000EC0A8AE2F80165850E94EC0A8EE6F80110
:1016900066850E94EC0A8FE6F80167850E94EC0AD5
:1016A00080E7F80160890E94EC0A81E7F80161890E
:1016B0000E94EC0A82E7F80162890E94EC0A1F91FD
:1016C0000F910895EF92FF920F931F93CF93DF93A3
:1016D0007B018C01603028E372072CE982072CE142
:1016E000920728F520E836E948E950E00E94A62F45
:1016F000E9016897B90180E090E020E839E647E623
:101700005FEF0E94742F6E0D7F1D801F911F32E0CE
:10171000660F771F881F991F3A95D1F721E732E0AE
:1017200040E050E00E94A62F890180E421C020E023
:101730003DE241E351E00E94A62FE9016897B9011B
:1017400080E090E020E033ED4EEC5EEF0E94742FDD
:101750006E0D7F1D801F911F660F771F881F991FB9
:1017600021E732E040E050E00E94A62F890180E6A8
:101770009E012F71622F680F85E70E94EC0A86E7B1
:10178000612F0E94EC0A87E7602F0E94EC0ACDB718
:10179000DEB7E6E00C940B3087E061E00E94EC0AD3
:1017A0008EE764E20E94EC0A88E063E00E94EC0AA3
:1017B00088E060E00E94EC0A87E065E00E94EC0AA5
:1017C00085E062E00E94EC0A83E00E94E60A8093D2
:1017D000F90384E00E94E60A8093FA030895582FE3
:1017E00040919E04842F90E0FC01EF70F0709F0107
:1017F0002F5F3F4F64E0959587956A95E1F728172D
:10180000390751F0E257FB4F5083842F8F5F8F7061
:10181000407F842B80939E0408951F920F920FB6F1
:101820000F9211241F932F933F934F935F936F93C6
:101830007F938F939F93AF93BF93CF93DF93EF9358
:10184000FF93C0918600D09187002091E0043091F1
:10185000E1048091BF04882309F062C0BE01621BCD
:10186000730B2091A1033091A2034091A3035091E7
:10187000A40325FD02C07695679589E0653C78074D
:10188000B8F180914703BCE1569547953795279568
:10189000BA95D1F7211531054105510521F421E013
:1018A00030E040E050E090E0A0E0B0E028173907D9
:1018B0004A075B07D0F4809147038F3FB1F020E0E7
:1018C0000EC0E22FF0E0EE0FFF1FDF01A054BB4F70
:1018D0008D919C91E95DFC4F918380832F5F809176
:1018E0004703281770F31092BE041092470318C0E4
:1018F00082E06D3B780760F180914703803140F5CD
:1019000010914703CB010E94160AE12FF0E0EE0F81
:10191000FF1FE054FB4F918380831F5F10934703A9
:10192000D093E104C093E004FF91EF91DF91CF9158
:10193000BF91AF919F918F917F916F915F914F91E7
:101940003F912F911F910F900FBE0F901F901895F0
:101950008FEF80934703E4CF83E0809380008AE990
:10196000809381008091A10386FD05C08091810054
:101970008064809381008FEF9FEF90938900809324
:10198000880080916F00806280936F0008956F30AF
:1019900018F086958058089589E0689F802D11245D
:1019A0000895882319F460E071E002C063E071E0FB
:1019B00087E396E00E94282D0895A0E0B0E0E3EED2
:1019C000FCE00C94ED2F182F0E94D9299B01AC014B
:1019D00080912D0590912E05A0912F05B091300595
:1019E00069017A01C81AD90AEA0AFB0AD701C601B5
:1019F00089589341A040B04010F010922C052093DC
:101A00002D0530932E0540932F05509330052091DE
:101A1000BF04822F81508230E8F580912C05882305
:101A200009F44FC1813011F482E0BCC1803108F06B
:101A300035C1E82FF0E0E054FB4F10838F5F8093B7
:101A40002C05803109F0B0C1A2ECB4E0213039F4AA
:101A50001196EC911197E695E6958C9109C08D91C0
:101A60009C911197E92FE695E695E69596958795D1
:101A7000E03140F4F0E090E0EE0FFF1FE95DFC4F35
:101A8000918380831092BE04129684E0A03DB80733
:101A9000E9F68AC1233009F004C180912C0588231E
:101AA00021F41F3009F080C10CC1883130F4E82FD7
:101AB000F0E0E154FB4F108374C1883109F0EEC0AF
:101AC000112309F0EBC0C0E0D0E00BE010E0DE0134
:101AD00063E0AA0FBB1F6A95E1F7C09FB001C19FE9
:101AE000700DD09F700D1124FB01E054FB4F8081DD
:101AF0002181922F977095958795FD01EE0FFF1F1D
:101B0000E95DFC4F91838083FB01EF53FB4F3081F4
:101B10003695369536952181422F4295440F407E69
:101B2000842F832B269526952695922F9770959531
:101B30008795FD01EE0FFF1FE75DFC4F91838083CA
:101B4000FB01EE53FB4F80818295869586958370CD
:101B50004181942F990F990F292F282B4295469553
:101B60004695437082818170880F880F382F342BFF
:101B700035952795FD01EE0FFF1FE55DFC4F318385
:101B80002083FB01EC53FB4F308136952181422F9E
:101B9000479544274795842F832B2695922F97703E
:101BA00095958795FD01EE0FFF1FE35DFC4F918337
:101BB0008083FB01EB53FB4F308132953F702181D5
:101BC000422F4295407F842F832B22952F70922F96
:101BD000977095958795FD01EE0FFF1FE15DFC4F16
:101BE00091838083FB01EA53FB4F8081881F882704
:101BF000881F4181942F990F292F282B441F442798
:101C0000441F82818370880F382F342B3595279598
:101C1000FD01EE0FFF1FEF5CFC4F31832083FB01C2
:101C2000E853FB4F3081369536952181422F4295FE
:101C3000440F440F407C842F832B26952695922FAA
:101C4000977095958795AA0FBB1FFD01ED5CFC4F22
:101C50009183808367537B4FFB01208122952695DA
:101C600027704181342F330F330F330F832F822B93
:101C7000942F92959695977095958795AB5CBC4FF0
:101C800011969C938E932196C230D10509F01FCFF7
:101C90008091D60483FD02C01092BE0410922C05E0
:101CA00083C0243009F080C040912C05442359F4AE
:101CB000183AB1F4109234051092330588EA0E9464
:101CC0005C0881E06FC0413019F41093310504C005
:101CD000423031F410933205812F0E945C085DC0C0
:101CE00060913205262F30E0220F331FE42FF0E001
:101CF000C90102968E179F0734F0433268F7E35408
:101D0000FB4F1083E9CF2D5F3F4F4091330550913A
:101D10003405E217F30749F4912F80E0482759274B
:101D2000509334054093330538C0812F90E0481715
:101D3000590789F580913105813069F5613118F0D5
:101D400080E180933205D090320540ECE42E44E0EF
:101D5000F42E00E010E01BC0F701D081C0E08181CB
:101D600090E08C2B9D2B33E0969587953A95E1F783
:101D70000E94160AF801EE0FFF1FE95DFC4F9183E8
:101D800080830F5F1F4F82E090E0E80EF91E0D1573
:101D900018F31092BE0410922C0580912C05882314
:101DA00019F08F5F80932C05CDB7DEB7E8E00C9477
:101DB0000930FF920F931F93CF93DF93182F092FB2
:101DC000F62E8EE30E94EC0A212F302FC901EC0180
:101DD00010E005C08FE769910E94EC0A1F5F1F1594
:101DE000C8F385E064E00E94EC0A83E00E94E60A02
:101DF0008093F90384E00E94E60A8093FA030E942C
:101E0000D9296093FB037093FC038093FD039093A7
:101E1000FE0387E069E00E94EC0A81E080939A0368
:101E2000CDB7DEB7E5E00C940C300E94D90E80915E
:101E30009A038130D9F40E94D9292091FB03309173
:101E4000FC034091FD035091FE03621B730B840B56
:101E5000950B605A76488140904040F4E8CF87E384
:101E600096E067E071E00E94282D089580919A0322
:101E70008130A9F3089587E396E06EE70E94E02E93
:101E80000895A0E0B0E0E7E4FFE00C94EC2F6C01D3
:101E900087E396E06EE70E94E02E7601C0E0D0E096
:101EA00000E010E0B0E2BB2E0AC00830110521F4BA
:101EB0009E012095F60120870894E11CF11CF70192
:101EC0006081862F8D57823040F487E396E06DE77E
:101ED0000E94E02EF70160816B2587E396E00E9467
:101EE000E02E0115110551F0F70180819E01280FA8
:101EF000311DC32FDD27C20FD31FD0700F5F1F4FBF
:101F00000930110591F6CDB7DEB7E9E00C94083041
:101F1000A9E0B0E0EEE8FFE00C94F32F382FE62FB5
:101F20008091A30490E0019664E270E00E94932FF8
:101F3000982F8093A30488E9898380E18A83913074
:101F400071F0913028F0923099F09330E1F416C09E
:101F500085E08B8381EF8C832F5F2D8317C09B835C
:101F600081EF8C8384E6489FC00111249D830EC0BD
:101F700084E08B8381EF8C833D8308C09B8381EF5A
:101F80008C83ED8303C00E943B0F04C0CE010196F9
:101F90000E94410F2996E2E00C940F300F931F939B
:101FA000CF93DF93182F092F87E396E06EE70E9407
:101FB000E02E212F302FC901EC0110E000E28881D2
:101FC0008D57823040F487E396E06DE70E94E02E63
:101FD00088818027888387E396E069910E94E02EBC
:101FE0001F5F193061F787E396E06EE70E94E02EED
:101FF000DF91CF911F910F910895A9E0B0E0E3E048
:10200000F0E10C94F32F382F8091A304882379F406
:102010008EEF89833A836B83842F90E09595879523
:102020008C832D83198618861F821E822FC04091B3
:102030009E04842F90E09C012F70307054E09595A1
:1020400087955A95E1F78217930721F18DEF8983E0
:102050001A821B82DE01149620E008C0E257FB4F73
:1020600080818D93405F2F5F263069F0842F90E050
:10207000FC0134E0F595E7953A95E1F78F709070A3
:10208000E817F90759F740939E042A83CE01019679
:102090000E94CE0F8091A30490E0019666E070E06C
:1020A0000E94932F8093A3042996E2E00C940F30B2
:1020B0009F92AF92BF92CF92DF92EF92FF920F93D7
:1020C0001F93B82EA62ED42EC22E902E0E94D92950
:1020D0007B018C0180918D0420919F043091A0049C
:1020E0004091A1045091A2048823B1F0D801C70106
:1020F000821B930BA40BB50B815E9E42A040B040A7
:1021000020F12C2DDC1408F42D2D8B2D6A2D422F5F
:10211000292D0E94880F11C0D801C701821B930B83
:10212000A40BB50B81539547A040B04070F08B2DA8
:102130006A2D4D2D2C2D0E94FD0FE0929F04F092F0
:10214000A0040093A1041093A2041F910F91FF908B
:10215000EF90DF90CF90BF90AF909F90089587E36E
:1021600096E0609100040E94E02E08951F93182FBE
:1021700087E396E0612F0E94E02E80910004812782
:10218000809300041F9108951F93192F0E94B61089
:10219000812F0E94B6101F910895DF92EF92FF9257
:1021A0000F931F93D82E7B011092000407E316E0D3
:1021B000C80165EB0E94E02EC80162E60E94E02E95
:1021C0008D2D0E94B610C7010E94C4101F910F915F
:1021D000FF90EF90DF900895E82FF0E0E456FC4F79
:1021E000E185E03148F4F0E0EE0FFF1FE95DFC4FC0
:1021F0000190F081E02D0DC0E03129F0E13129F0AE
:10220000E0E0F2E006C082E101C083E10E942D2BF4
:10221000FC01CF0108958CE060E00E945E2A8BE013
:1022200061E00E945E2A8DE061E00E945E2A82E009
:1022300060E00E945E2A84E061E00E945E2A0895C8
:1022400082E08093B00085E08093B10083E061E09C
:102250000E945E2A83E060E00E94CA2A08951F93CC
:10226000182F0E94D92960939F047093A004809333
:10227000A1049093A20410938D04112329F440E843
:1022800055E260E070E004C040E051EE60E070E0D4
:1022900087E396E00E94E62D1F91089583E00E9457
:1022A000E60A8093F90384E00E94E60A8093FA0329
:1022B00087E061E00E94EC0A6AE070E080E090E074
:1022C0000E94FF290E94CC0B000008959F92AF92BC
:1022D000BF92CF92DF920F93DF93CF9300D000D0C5
:1022E000CDB7DEB7982E89E061E00E94CA2A62E38A
:1022F00070E080E090E00E94FF2989E060E00E94A9
:10230000CA2A62E370E080E090E00E94FF2983E047
:102310000E94E60A8093F90384E00E94E60A809313
:10232000FA0386E060E00E94EC0A87E061E00E9428
:10233000EC0A89E06FE70E94EC0A8AE065E00E94FF
:10234000EC0A8BE065E10E94EC0A8CE062E10E94FD
:10235000EC0A8DE06DEF0E94EC0A8EE060E00E94D6
:10236000EC0A992019F084E193E008C08091F7030A
:1023700023E1829FC00111248B549D4F0E94110BB9
:1023800080E36CE80E94EC0A82E36FE00E94EC0AB2
:1023900083E362E40E94EC0A84E36AE00E94EC0AB0
:1023A00085E36AE20E94EC0A86E36DE20E94EC0A91
:1023B00087E364ED0E94EC0A88E360E00E94EC0A87
:1023C00089E360E00E94EC0A992049F0A5E8AA2E72
:1023D000A1ECBA2EA1ECCA2EAEEDDA2E08C0A09068
:1023E000D903B090DA03C090DB03D090DC030AE39A
:1023F0008D2D9927AA27BB2789839A83AB83BC831A
:10240000802F69810E94EC0A802F8B5F69810E9476
:10241000EC0ADC2CCB2CBA2CAA240F5F0E3341F72C
:1024200083E46FEF0E94EC0A84E46FEF0E94EC0AF1
:1024300085E46FEF0E94EC0A86E46FEF0E94EC0ADD
:10244000992019F08DE666E003C08DE66091DD030A
:102450000E94EC0A89E760E00E94EC0A8AE760913A
:10246000DE030E94EC0A83E760E00E94EC0A84E746
:1024700060E00E94EC0A992029F060EC7AEC89E88F
:1024800096E308C06091D5037091D6038091D7037D
:102490009091D8030E94620B0F900F900F900F90B5
:1024A000CF91DF910F91DF90CF90BF90AF909F9031
:1024B0000895A0E2B0E0EFE5F2E10C94EB2F8CE0A0
:1024C0000E94E60A882379F587E396E063E171E0EC
:1024D0000E94282D5E9A80E00E9466110E94CC0B1B
:1024E0005E9821C087E396E00E94A72E482F809136
:1024F000BF04882321F0842F0E94DD0C14C080913A
:102500002A05E82FF0E031969F012F713070319746
:102510008091290590E02817390729F0E050FB4FFA
:10252000408320932A0587E396E00E946D2E892B35
:10253000C9F680919A03843009F08EC00E94D9298F
:102540006093AE047093AF048093B0049093B10491
:10255000611571058105910561F481E090E0A0E0CD
:10256000B0E08093AE049093AF04A093B004B09316
:10257000B1048091BA049091BB0481609093BB0434
:102580008093BA0483E080939A038FE70E94C20A83
:1025900007EF14E00E94D60AF80181938F01F5E05D
:1025A00000301F07B9F74091E2048091F704282F0B
:1025B00030E0842F90E08227932786FF40C080E49C
:1025C00048274093E204C90188739070C89709F5C1
:1025D00010E014C01F5F8091F803E12FF0E084FF4A
:1025E00006C0E950FB4F80810E94EF0B07C0E95005
:1025F000FB4F87E396E060810E94E02E212F30E0C0
:102600008091F70490E0877090708217930714F719
:1026100016C02F733070232B91F48091F8048093AF
:10262000B2048091F9048093B4048091FA048093F9
:10263000B5048091FD048093BC041092BD04809188
:102640002B05813019F482E080932B0580912B05B6
:10265000833011F410922B050E94D9295B016C0183
:102660008091B6049091B704A091B804B091B904D8
:102670000097A105B105C9F086017501E81AF90AAC
:102680000A0B1B0BD801C701885B9B40A040B040E0
:1026900060F00E940D0B8093B3041092B604109268
:1026A000B7041092B8041092B90480ED93E00E9430
:1026B00021092091AA043091AB044091AC045091BF
:1026C000AD0486017501E21AF30A040B150BE61638
:1026D000F7060807190708F40DC1A092AA04B092E2
:1026E000AB04C092AC04D092AD04A8958091BE0416
:1026F0008830A0F08091A1039091A203A091A30340
:10270000B091A4032CE1B695A795979587952A9546
:10271000D1F70097A105B10509F08BC18091BE04E6
:102720008F5F8093BE04E090AE04F090AF04009100
:10273000B0041091B104E114F1040105110511F187
:1027400080ED93E00E942109AE18BF08C00AD10AAB
:102750006A157B058C059D0588F48091A10384FD95
:1027600004C080ED97E00E940C081092AE04109215
:10277000AF041092B0041092B10404C080E090E065
:102780000E940C089091E204907C9093E2040091E6
:102790002A05109129050117B1F180912B0582308E
:1027A00091F590589093E20480ED93E00E94170910
:1027B000893010F048E002C0482F415030E013C08B
:1027C0003F5FA32FB0E0812F90E0FC01E050FB4F72
:1027D0002081FD01EE51FB4F2083A05EBA4F2C9368
:1027E0000196182F1F71341710F4101749F7109322
:1027F0002905832F895C9091E204892B8093E20460
:10280000309320051AC020912B052430D1F49091EB
:102810002005E1E2F5E0A3EEB4E0292F30E02E0F31
:102820003F1F02C081918D93E217F307D9F7995C9E
:102830008091E204982B9093E20483E080932B052F
:1028400037C08091A504823029F491609093E2040E
:102850005E9A0FC09093E2045E98222319F481E0FF
:1028600080932B0580912B05833019F484E08093AD
:102870002B05F89405EA13E07E010894E11CF11C95
:10288000F80181918F010E94EC10F70181939193DF
:102890007F01F3E0053B1F0799F78091F8038770EC
:1028A000BE016F5F7F4F43EE54E00E94A809789409
:1028B0005D9A8091A4040E94F70A80ED93E00E9443
:1028C0001709682F82EE94E00E94D90EE091A404CB
:1028D000EF5FE093A404E83131F0F0E0E053FC4F07
:1028E0008785882339F41092A40404C05E9A89E095
:1028F0008093BE048091F803887171F180919A03EE
:10290000823051F58091BA049091BB04880F991FD1
:102910009093BB048093BA0483E080939A030E944F
:10292000CC0B0E94D9296093B6047093B7048093AE
:10293000B8049093B904611571058105910561F49E
:1029400081E090E0A0E0B0E08093B6049093B704FB
:10295000A093B804B093B9048091F80384FF1EC01B
:102960008091BA049091BB048E7F0E946A0A182F4E
:102970008091B2046091BC040E94C70C082F809122
:10298000B304612F0E94C70C282F8091B40460917A
:10299000B504402F00919B030E9458105D988091D0
:1029A000A5048130D1F0813020F0823009F047C099
:1029B00034C08EE00E94FD2A892B09F040C081E0DE
:1029C0008093A5040E94CB296093A6047093A7046A
:1029D0008093A8049093A90432C08EE00E94FD2A3F
:1029E000892B21F50E94CB292091A6043091A704C0
:1029F0004091A8045091A904621B730B840B950BA2
:102A0000695E734080409040D0F082E08093A504DE
:102A100080ED97E00E940C0812C08EE00E94FD2A13
:102A2000892B69F080E090E00E940C081092A504C8
:102A300006C08091BE04883009F059CF57CFA096C8
:102A4000EAE00C940730ACE1B0E0E9E2F5E10C9487
:102A5000EB2F0E94D9297B018C0181E00E94661135
:102A600054E7A52E6E010894C11CD11C43E0B42E7E
:102A7000A982C60161E00E94150FB0929A030E94DC
:102A8000CC0B6AEF70E080E090E00E94FF2980911B
:102A90009A03833009F07DC087E396E00E946D2E93
:102AA000892B09F076C00E94D9296E197F09800B05
:102AB000910B6058734C894C914008F06AC0D8CF94
:102AC0008FE70E94C20A0E94D60A843509F05CC0D2
:102AD00089830E94D60A182F00E010938C0400937B
:102AE0008B040E94D60A080F111D10938C040093CA
:102AF0008B040E94D60A80938A040E94D60A80938F
:102B00008904813108F040C0FF2407C00E94D60A22
:102B100007591B4FF8018083F3940F2D10E080912B
:102B2000890490E0880F991F0817190778F380E748
:102B30008983CE01019661E00E94150F83E08093A6
:102B40009A030E94CC0B62E370E080E090E00E9468
:102B5000FF2980919A038330A9F08FE70E94C20A6F
:102B60000E94D60A803581F4898305EB13E00E9428
:102B7000D60AF80181938F01F3E0003D1F07B9F7F2
:102B800081E003C082E001C083E06C96EAE00C942F
:102B9000073080919A03833009F092CFF3CF0F93DF
:102BA0001F93082F17C05E9A64E670E080E090E003
:102BB0000E94FF295E9864E670E080E090E00E9449
:102BC000FF291F5F101778F36CE271E080E090E05E
:102BD0000E94FF2910E0F6CF482F392F25E00DC0C5
:102BE000F999FECF1FBA842F932F92BD81BD60BD8E
:102BF0000FB6F894FA9AF99A0FBE215059F0F99944
:102C0000FECF842F932F92BD81BDF89A80B56817AF
:102C100039F7089582E00E94CF150895A0E0B0E052
:102C2000E4E1F6E10C94E42F482E562EEE24FF2426
:102C300088249924C0E0D0E0CC24DD2416E4312E91
:102C400004C055245394CC24DD24442069F480919D
:102C50009B03839DE0011124BCE9EB2EB3E0FB2E26
:102C6000A9E18A2E912C1DC021E0421671F48091B9
:102C70009B03839DE00111246B96F0EDEF2EF3E0B2
:102C8000FF2EE9E28E2E912C0CC032E0431649F45F
:102C90007BE9E72E73E0F72E61E0862E912CC8E1E8
:102CA000D1E03E016C0C7D1C10923405109233056E
:102CB000E3011BC0552059F4F999FECFD2BDC1BD27
:102CC000F89A80B5F701E00FF11F808307C0F70184
:102CD000E00FF11FCE0160810E94EC150E0D1F1D4B
:102CE000F80180810E945C0821969E012619022F1E
:102CF00010E008151905F0F2CE015520D9F4F99924
:102D0000FECFD2BDC1BDF89A20B5F999FECF21966C
:102D1000D2BDC1BD2197F89A80B590E0B22EAA2409
:102D20008A299B29209133053091340528173907CA
:102D300059F487CF2196609134050E94EC15CE019D
:102D4000609133050E94EC1580E291E0C80ED91E17
:102D500091EEC91692E0D90608F477CF852DCDB74C
:102D6000DEB7E1E10C94003080E061E00E940E16D5
:102D700081E061E00E940E16089580E060E00E940C
:102D80000E16882331F081E060E00E940E16882341
:102D900031F40E94BE080E9479080E94B41608957A
:102DA00082E061E00E940E16089582E060E00E94D9
:102DB0000E1680919B03843020F010929B030E949A
:102DC000D01608951F93182F0E94D51680919B034B
:102DD000811731F0143020F410939B030E94D01619
:102DE0001F9108951092670485E6E2E0F4E0DF01A8
:102DF0001D928A95E9F708951F93182F8F3711F0C8
:102E00008830E1F5E0916704EE2309F455C0E15004
:102E1000E0936704F0E0EE5FFB4F108287E396E0FB
:102E20006DE00E94E02E10E00AC0E12FF0E0EE5FBE
:102E3000FB4F87E396E060810E94E02E1F5F809148
:102E40006704181790F387E396E060E20E94E02E93
:102E500087E396E06DE00E94E02E10E00AC0E12FCB
:102E6000F0E0EE5FFB4F87E396E060810E94E02E8A
:102E70001F5F80916704181790F31CC08B3119F401
:102E80000E94F2161FC08D30E9F08A30D9F080918F
:102E90006704843688F487E396E0612F0E94E02E71
:102EA00080916704E82FF0E0EE5FFB4F10838F5FA7
:102EB0008093670480E007C087E396E067E00E94A4
:102EC000942BF8CF81E01F9108951F93CF93DF9348
:102ED000CFEDD3E010E03BC087E396E062E271E023
:102EE0000E94252D87E396E0612F4AE050E00E9482
:102EF000A22C87E396E06FE271E00E94252D699194
:102F000070E080E090E02091DE0330E040E050E0AF
:102F10000E94742F20E137E240E050E00E94742FBD
:102F2000DC01CB014091D5035091D6036091D703CA
:102F30007091D803480F591F6A1F7B1F87E396E0E3
:102F40002AE030E00E94692C1F5F183119F0888157
:102F5000882311F6DF91CF911F910895EF92FF9290
:102F60000F931F93882339F487E396E061E77AE0B3
:102F70000E94B22B3BC090E00E94DE0824E630E0C5
:102F800040E050E00E94A62F122F032FF42EE52ED2
:102F9000622F732F842F952F2AE030E040E050E01D
:102FA0000E94A62F87E396E0BA01A9012AE030E04B
:102FB0000E945A2C87E396E06EE20E94942B612FC8
:102FC000702F8F2D9E2D2AE030E040E050E00E94CF
:102FD000A62FAB01BC0187E396E02AE030E00E9417
:102FE0005A2C87E396E063E70E94C62B1F910F914E
:102FF000FF90EF900895FF920F931F93CF93DF936D
:1030000087E396E067E67AE00E94732B8091B50330
:10301000813041F487E396E06EE47AE00E94B22BBF
:10302000FF246DC0823029F487E396E067E37AE0FD
:10303000F5CF843029F487E396E063E27AE0EECFBF
:10304000853071F787E396E068E17AE0E7CFCF2D2E
:10305000D0E0C930D1051CF06F2D685C02C06F2D27
:103060006F5C87E396E00E94942B87E396E060E133
:103070007AE00E94732BBE016F5F7F4F87E396E07B
:103080004AE050E00E94FE2C87E396E065E07AE09B
:103090000E94732B8E010B541C4FD8011196EC919A
:1030A000E032F8F487E396E068EF79E00E94732B52
:1030B000F8018181803130F087E396E063E371E0CD
:1030C0000E94252DCB54DC4F698170E06F707070C9
:1030D0006F5F7F4F87E396E04AE050E00E94112D3A
:1030E0000DC0F0E0EF70F070EE0FFF1FE75BFC4FDC
:1030F0006081718187E396E00E94282DF39480918E
:103100008A04F81608F4A3CF87E396E06DED79E022
:103110000E94732B8091CD030E94AE1787E396E047
:1031200062EC79E00E94732B8091CE030E94AE176F
:1031300087E396E067EA79E00E94732B8091CF03E2
:103140000E94AE1787E396E06CE879E00E94732B4B
:103150004091C5035091C6036091C7037091C803A5
:10316000411551056105710539F187E396E02AE0C3
:1031700030E00E94692C87E396E069E579E00E94DF
:10318000732B8091C9030E941109AB01BC0187E335
:1031900096E02AE030E00E94692C87E396E065E340
:1031A00079E00E94732B87E396E06091CA034AE0BE
:1031B00050E00E94B42C06C087E396E06CE279E010
:1031C0000E94B22B87E396E06FE079E00E94732BB8
:1031D0006091CB037091CC0387E396E04AE050E026
:1031E0000E948E2C87E396E062EF78E00E94732BBA
:1031F0006091C403603150F470E06F5F7F4F87E3EC
:1032000096E04AE050E00E94112D06C087E396E068
:1032100069EE78E00E94B22B87E396E06CEC78E0F0
:103220000E94732B8091C30380FD03C065E371E0AE
:1032300002C069E371E087E396E00E94282D87E3EE
:1032400096E06FEA78E00E94732B8091C30382704E
:103250000E94D10C87E396E060E978E00E94732B2E
:103260008091C30384700E94D10C87E396E061E7EC
:1032700078E00E94732B8091C30388700E94D10C68
:10328000CDB7DEB7E5E00C940C301F93CF93DF93FE
:1032900087E396E06BEB7BE00E94732B4091D503B4
:1032A0005091D6036091D7037091D80387E396E0DD
:1032B0002AE030E00E94692C87E396E065EA7BE033
:1032C0000E94732B4091D9035091DA036091DB0384
:1032D0007091DC0387E396E020E130E00E94692CE6
:1032E00087E396E06FE87BE00E94732B87E396E02C
:1032F0006091DD034AE050E00E94B42C87E396E041
:1033000069E77BE00E94732B87E396E06091DE0320
:103310004AE050E00E94B42C87E396E063E67BE04D
:103320000E94732BCFEDD3E010E012C0112331F0D7
:1033300087E396E06DE371E00E94252D87E396E038
:1033400069914AE050E00E94A22C1F5F183119F0E9
:103350008881882359F787E396E00E949C2B87E3B6
:1033600096E06DE47BE00E94732B87E396E060912A
:10337000F7034AE050E00E94B42C87E396E068E34C
:103380007BE00E94732BE091F803F0E0E770F070AF
:10339000EE0FFF1FE759FC4F6081718187E396E0D4
:1033A0000E94282D87E396E063E27BE00E94732B66
:1033B0008091F80390E0887190708830910589F0D1
:1033C000893091051CF4892B39F01BC0803191059F
:1033D00069F04897B1F40FC087E396E06AE17BE0BB
:1033E0000EC087E396E06EE07BE009C087E396E0DD
:1033F00068E07BE004C087E396E06EEF7AE00E942D
:10340000B22B87E396E06AEE7AE00E94732B40913C
:10341000D1035091D2036091D3037091D40387E319
:1034200096E02AE030E00E94692C87E396E061EDA7
:103430007AE00E94732B8091A10380710E94D10CCD
:1034400087E396E068EB7AE00E94732B8091A103FA
:1034500080740E94D10C87E396E06FE97AE00E94C5
:10346000732B8091A10380720E94D10C87E396E0B8
:1034700062E87AE00E94732B80ED93E00E942109BC
:10348000AB01BC0187E396E02AE030E00E945A2CB1
:1034900087E396E06DE77AE00E94732B80ED93E07E
:1034A0000E9421099B01AC0160E472E48FE090E08E
:1034B0000E94A62F87E396E0BA01A9012AE030E036
:1034C0000E945A2C87E396E06AE77AE00E94B22BCA
:1034D000DF91CF911F910895EF92FF920F931F9369
:1034E0008C0137E3E32E36E0F32EC701612F70E045
:1034F0004AE050E00E947D2CC7016EE20E94942BAE
:1035000024E0169507952A95E1F70F701070C70112
:10351000B8014AE050E00E947D2C1F910F91FF906E
:10352000EF9008950F931F93CF93DF9320910104A1
:103530002F3FA9F587E396E061EF75E00E94732BBA
:1035400080E793E00E946C1A87E396E060ED75E0F7
:103550000E94732B80918B0490918C040E946C1AB2
:1035600087E396E06DE975E00E94B22B87E396E071
:103570006AE775E00E94B22B87E396E062E675E0A9
:103580000E94B22B87E396E06DE375E00E94B22BB8
:1035900087E396E00E949C2B0E94FB1769C01216DD
:1035A0000CF066C0332727FD309580918A0490E0A7
:1035B000821793070CF45CC087E396E068E275E03D
:1035C0000E94732B60910104772767FD709587E354
:1035D00096E04AE050E00E94112D87E396E06DEFFF
:1035E00074E00E94732B08E210E03AC0C12FD0E0D3
:1035F000CC0FDD1FC759DB4F288130E080910104DB
:10360000992787FD909501972817390741F587E39A
:1036100096E06FE371E00E94252D87E396E0602F2E
:103620004AE050E00E94A22C87E396E063E471E058
:103630000E94252DE981F0E0EF70F070EE0FFF1F82
:10364000E75BFC4F6081718187E396E00E94252D46
:1036500087E396E067E471E00E94252D0F5F1F5F0E
:1036600080918904181710F287E396E00E949C2B42
:10367000DF91CF911F910F910895ACE1B0E0E3E4A9
:10368000FBE10C94ED2F282F809101048F3F09F06E
:1036900042C1822F90E0FC013A97EF36F10508F025
:1036A00033C1EC5CFF4F0C941A3087E396E069E479
:1036B00071E0AEC087E396E069E471E00E94282DD6
:1036C0001CC187E396E065E571E00E94282D85E73F
:1036D0008983DE011296E5EBF3E08BE101900D9218
:1036E0008150E1F7CE0101966CE10E94150F0E9416
:1036F000CC0B83E080939A0368EC70E080E090E06C
:103700000E94FF2980919A03843009F0FDC08FE761
:103710000E94C20A0E94D60A8983853509F0F4C046
:1037200087E396E06FED74E00E94B22B87E396E0AA
:1037300061EC74E00E94B22B87E396E063EA74E0E8
:10374000ACC087E396E06DE671E00E94282D89E623
:103750008983CE01019661E00E94150F0E94CC0B77
:1037600083E080939A0368EC70E080E090E00E9430
:10377000FF2980919A03843009F0C6C08FE70E9428
:10378000C20A0E94D60A89838E010E5F1F4FBDE1D7
:10379000EB2EF12CEC0EFD1E0E94D60AD8018D9363
:1037A0008D01AE15BF05C1F7A5EBB3E0FE01329662
:1037B0008BE101900D928150E1F78981893409F004
:1037C000A3C087E396E065E874E00E94B22B87E32C
:1037D00096E067E674E00E94B22B87E396E069E426
:1037E00074E05BC087E396E067E871E00E94282DF3
:1037F0008EEF8093010488C020522750922F90535F
:1038000080918A04891738F487E396E066E971E0CD
:103810000E94282D79C0909301046FC084E18093A9
:10382000010487E396E062E174E037C085E18093AC
:10383000010487E396E06BED73E02FC086E180938F
:10384000010487E396E064EA73E027C087E1809390
:10385000010487E396E06AE573E01FC088E1809386
:10386000010487E396E069E473E017C089E180937F
:10387000010487E396E065E373E00FC08AE180937B
:10388000010487E396E060E273E007C08BE1809378
:10389000010487E396E068EF72E00E94B22B34C027
:1038A00087E396E06EED72E00E94B22B8091C30335
:1038B00091E01DC087E396E068EC72E00E94B22BB5
:1038C0008091C30392E013C087E396E063EB72E05C
:1038D0000E94B22B8091C30394E009C087E396E075
:1038E00068E972E00E94B22B8091C30398E08927B7
:1038F0008093C3038FEF809301040E94921A04C047
:1039000087E396E00E94A72E87E396E00E946D2E43
:10391000892BB1F762C1822F0E94FC16882309F41B
:103920005CC180916704882321F48FEF80930104A8
:103930004CC182E094E060E070E040E050E00E9422
:10394000A2069B01AC0160910104862F992787FD97
:103950009095A92FB92FFC013197EB31F10508F0B3
:1039600024C1ED55FF4F0C941A30E62FFF27E7FDD9
:10397000F09580918A0490E08E179F070CF415C192
:10398000DA01C9010197A109B1098097A105B10523
:1039900048F0A8E2FA2E00E010E06F010894C10898
:1039A000D10825C0EB54FC4F822F81508083E5C0A5
:1039B000612F70E0660F771F67597B4FFB01808195
:1039C00090E08C159D0591F48F2D90E0A0E0B0E083
:1039D00082179307A407B50741F4F601EB54FC4F97
:1039E000DB0111968C91818301E0F3941F5F80913C
:1039F00089041817E8F2BFC02F3F31054105510572
:103A000011F008F0D2C02093CD03B7C02F3F31058D
:103A10004105510511F008F0C8C02093CE03ADC098
:103A20002F3F31054105510511F008F0BEC020932C
:103A3000CF03A3C0809102048062803719F583E030
:103A400094E060E070E040E050E00E94A2069B013C
:103A5000AC01DC01CB010197A109B1090897A105CF
:103A6000B10508F0B5C0CA01B90124ED30E340E06A
:103A700050E00E94742F9B01AC012A5E3C4A4A46EA
:103A8000554E24C0863611F583E094E060E070E086
:103A900040E050E00E94A2069B01AC01DC01CB019A
:103AA0000197A109B1090797A105B10508F090C0D8
:103AB000CA01B90128EA31E640E050E00E94742FC3
:103AC0009B01AC01245E3C434E46544E211531050A
:103AD0004105510561F0DA01C901805C9D49A845A5
:103AE000B54381509A45A246B24008F05EC020938B
:103AF000C5033093C6034093C7035093C8033DC02A
:103B00002F3F31054105510511F008F04EC02093BB
:103B1000C90333C0DA01C9010197A109B1098F3F77
:103B20009105A105B10508F040C02093CA0325C046
:103B3000DA01C901845C9940A040B0408D549D4198
:103B4000A040B04030F43093CC032093CB0301E08D
:103B500001C000E0211531054105510511F48FEF39
:103B600007C0213131054105510528F4822F8150CC
:103B70008093C40302C00023C1F0809168048823AD
:103B8000D1F48091D9039091DA03A091DB03B09135
:103B9000DC030196A11DB11D8093D9039093DA0334
:103BA000A093DB03B093DC0306C087E396E068EAEA
:103BB00071E00E94282D0E94F2168FEF809301047D
:103BC00087E396E06AE00E94C62B0E94921A05C025
:103BD00021E030E040E050E07ECF6C96E8E00C94CD
:103BE000093087E396E06CE472E00E94B22B87E331
:103BF00096E064E372E00E94B22B87E396E00E94B5
:103C00006D2E892B31F087E396E00E94A72E0E944B
:103C10003D1B0E942315823019F0833069F405C0E2
:103C200087E396E066E172E004C087E396E06FEF19
:103C300071E00E94B22B08958FEF809301041092DF
:103C400068040E94921A0CC087E396E00E946D2ED1
:103C5000892B31F087E396E00E94A72E0E943D1B3E
:103C6000809101048E3F81F7089580910104992786
:103C700087FD9095A92FB92FFC013196EB30F10506
:103C800008F074C0E254FF4F0C941A3087E396E0BA
:103C900064E678E00E94B22B80E793E00E946C1A01
:103CA00087E396E06CE478E00E94B22B87E396E02D
:103CB00067E278E00E94B22B87E396E06DEF77E051
:103CC0000E94B22B87E396E06CED77E00E94B22B66
:103CD00087E396E06FEA77E00E94B22B87E396E0F5
:103CE00069E877E00E94B22B87E396E065E677E02B
:103CF0000E94B22B87E396E06EE377E00E94B22B3E
:103D000087E396E00E949C2B0E9445192FC087E311
:103D100096E061E277E028C087E396E06CEF76E01A
:103D200023C087E396E067EE76E01EC087E396E067
:103D300068EC76E019C087E396E064E876E014C0AA
:103D400087E396E06FE676E00FC087E396E06AE5EA
:103D500076E00E94B22B87E396E064E176E004C04F
:103D600087E396E06EEF75E00E94B22B6AE070E0A8
:103D700080E090E00E94FF2904C087E396E00E9463
:103D8000A72E87E396E00E946D2E892BB1F7089548
:103D9000A2E2B0E0EEECFEE10C94E32F8E010F5FA7
:103DA0001F4F80E1D8011D928A95E9F787E396E0DD
:103DB00066EC71E00E94282D0E944E1120EC3DE936
:103DC00048E555E32F8F38A349A35AA380EC97EF1A
:103DD000AAEBB7E38B8F9C8FAD8FBE8F24EF31E0C2
:103DE00040E050E02F8B388F498F5A8F30E5C32E3B
:103DF00033ECD32EE12CF12C20EC422E2DE9522E67
:103E000028E5622E25E3722E882499245401332458
:103E10001E8A1D8A198A1A8A1B8A1C8AFFC087E398
:103E200096E00E94A72E8434B9F0853430F48332B2
:103E3000B9F18C3209F0CCC044C0833509F0C8C058
:103E40002F8D38A149A15AA1C901DA012C013D01E8
:103E5000882499245401E2C087E396E064E40E9438
:103E6000942B87E396E040EC5DE968E575E32AE092
:103E700030E00E94C82C87E396E06CE20E94942B0D
:103E800087E396E040EC57EF6AEB77E32AE030E017
:103E90000E94C82C87E396E06CE20E94C62BBEC04D
:103EA00019821A821B821C821D821E821F82188622
:103EB00019861A861B861C861D861E861F86188AF2
:103EC0003AC0339434E0331609F0A8C069817A818E
:103ED0008B819C8128EE33E040E050E00E94742FFB
:103EE0006F8F78A389A39AA36D817E818F81988536
:103EF0000E94742F6B8F7C8F8D8F9E8F89859A8502
:103F0000AB85BC858F8B988FA98FBA8F6D857E8589
:103F10008F8598890E94742F6B017C0190E2C916ED
:103F20009EE4D90690E0E90690E0F90630F48CE1D1
:103F300062E30E94EC0A332471C0A0E3CA16A5E72D
:103F4000DA06A0E0EA06A0E0FA0618F48CE162E2E4
:103F5000F0CFB0E4CB16BCE9DB06B0E0EB06B0E096
:103F6000FB0618F48CE166E2E4CFE0E5CE16E3EC64
:103F7000DE06E0E0EE06E0E0FE0618F48CE162E129
:103F8000D8CFF0E6CF16FAEEDF06F0E0EF06F0E06D
:103F9000FF0618F48CE165E1CCCF20E7C21621E1E1
:103FA000D20621E0E20620E0F20618F48CE161E09E
:103FB000C0CF30EAC31636E8D30631E0E30630E07E
:103FC000F30618F48CE163E0B4CF8CE165E0B1CF87
:103FD00090ED292E280E49E0421500F1032D10E046
:103FE000000F111F000F111F81E090E08C0F9D1F2B
:103FF000080F191FD8016D917D918D919C912AE038
:1040000030E040E050E00E94742F620D711D811D70
:10401000911DF801608371838283938387E396E027
:104020000E946D2E892B09F0FACE81149104A1040F
:10403000B10489F4C301B2010E94620B61E070E037
:1040400080E090E00E94FF29FFEFFE8B1D8A198A15
:104050001A8A1B8A1C8A2F89388D498D5A8D82169F
:104060009306A406B506E0F40E940D0B29893A894F
:104070004B895C89280F311D411D511D298B3A8BBD
:104080004B8B5C8B3D89381708F48D8B4E898417D8
:1040900008F48E8B0894811C911CA11CB11C56C085
:1040A000C301B20128EE33E040E050E00E94A62FA9
:1040B00087E396E0BA01A9012AE030E00E945A2C79
:1040C00087E396E06CE20E94942B87E396E06D898B
:1040D0004AE050E00E94A22C87E396E06CE20E9446
:1040E000942B69897A898B899C89A50194010E9406
:1040F000A62F87E396E0BA01A9012AE030E00E94EA
:104100005A2C87E396E06CE20E94942B87E396E0BA
:104110006E894AE050E00E94A22C87E396E06CE2B0
:104120000E94C62B4C0C5D1C6E1C7F1C8B8D9C8DC5
:10413000AD8DBE8D84159505A605B70520F44F8C71
:1041400058A069A07AA08824992454012F8D38A101
:1041500049A15AA1285E33404040504009F05ECF4B
:10416000A296E2E10C94FF2FAAE5B0E0EAEBF0E2C0
:104170000C94EF2F8B017A018B3009F426C18C301F
:1041800040F5853009F484C0863080F4823009F42B
:1041900059C0833020F4813009F052C242C08330CC
:1041A00009F461C0843009F04BC265C0883009F45D
:1041B0009DC0893038F4863009F486C0873009F014
:1041C0003FC28CC0893009F499C08A3009F038C2E6
:1041D000C9C0893609F484C18A3680F4863609F468
:1041E0002FC1873620F4853609F02AC210C18736E0
:1041F00009F43FC1883609F023C243C18C3609F463
:10420000C6C18D3638F48A3609F475C18B3609F08B
:1042100017C2B1C18D3609F4EEC1873C09F010C256
:1042200002C281E069E270E00E94CD1000ED13E06F
:10423000F80181918F010E94B610F3E0093F1F073A
:10424000B9F706C282E06BE170E00E94CD1005EB89
:1042500013E0F80181918F010E94B610F3E0003D58
:104260001F07B9F7F5C183E061E070E00E94CD104F
:104270000E942315EBC184E061E070E00E94CD1044
:1042800081E00E94B6100E94AF100E94C81EE2C1D9
:104290006091890470E0660F771F85E00E94CD1061
:1042A00000E010E008C0F801E759FB4F80810E9450
:1042B000B6100F5F1F4F8091890490E0880F991FFF
:1042C0000817190780F3C4C186E062E070E00E941D
:1042D000CD1080E793E00E94C410BAC187E061E08E
:1042E00070E00E94CD1080918A04B0C188E061E046
:1042F00070E00E94CD1080919B03A8C186E689835F
:10430000CE01019661E00E94150F0E94CC0B83E064
:1043100080939A0368EC70E080E090E00E94FF29AF
:1043200080919A038430E1F48FE70E94C20A0E94D0
:10433000D60A8983863471F489E060E270E00E94D5
:10434000CD1010E00E94D60A0E94B6101F5F1032F6
:10435000C9F77EC189E061E070E00E94CD10C9C05C
:1043600089E06FC18AE069E170E00E94CD1082E0CF
:1043700080939C038091A105882351F08091A10333
:104380009091A203A091A303B091A403806809C0F7
:104390008091A1039091A203A091A303B091A403E3
:1043A0008F778093A1039093A203A093A303B0936C
:1043B000A4030CE913E0F80181918F010E94B6106B
:1043C000F3E0053B1F07B9F743C18BE061E270E002
:1043D0000E94CD108091BE048F3F39F08091BE04C1
:1043E0008F5F8093BE04815002C08091BE040E9402
:1043F000B61010E0F894812F0E94EC100E94450A3C
:104400000E94C41078941F5F1031A1F721C185E686
:1044100061E070E00E94CD100932110509F015C16C
:1044200020E030E0F901E053FC4FD701A20FB31FA9
:104430008C9180832F5F3F4F2932310599F759C006
:1044400086E661E070E00E94CD100B31110509F0A5
:10445000FCC020E030E0F901EB54FC4FD701A20F83
:10446000B31F8C9180832F5F3F4F2B31310599F71C
:1044700040C087E661E070E00E94CD100E94B41653
:1044800038C088E661E070E00E94CD1085E78A833D
:10449000DE011396E5EBF3E08BE101900D92815084
:1044A000E1F7CE0102966CE10E94150F0E94CC0B41
:1044B00083E080939A0360E273E080E090E00E94E2
:1044C000FF2980919A03843009F0BFC08FE70E94D2
:1044D000C20A0E94D60A8A83853509F0B6C009C08F
:1044E00089E661E070E00E94CD100E9479080E9488
:1044F000BE0881E0ABC08AE661E070E00E94CD10AA
:1045000089E68E8FCE014E9661E00E94150F0E94C3
:10451000CC0B83E080939A0360E273E080E090E04C
:104520000E94FF2980919A03843009F08EC08FE7A2
:104530000E94C20A0E94D60A8E8F8E01015E1F4F12
:104540004AE3E42EF12CEC0EFD1E0E94D60AF8017F
:1045500081938F01EE15FF05C1F7A5EBB3E0FE01D6
:104560007F968BE101900D928150E1F78E8D893419
:1045700009F06BC0BECF8BE661E070E00E94CD1009
:10458000F70180810E94E2160E94BD16B2CF8CE630
:1045900061E070E00E94CD100032110571F487E6F1
:1045A0008AAFDE01DB96F70180E201900D92815027
:1045B000E1F7CE01CA9661E205C087E48AAFCE0179
:1045C000CA9661E00E94150F0E94CC0B83E0809395
:1045D0009A036CE474E080E090E00E94FF298091EF
:1045E0009A03843091F58FE70E94C20A0E94D60A8E
:1045F000873459F57ECF8DE661E070E00E94CD10E2
:104600000931110511F520E030E0F901E456FC4FC5
:10461000D701A20FB31F8C9180832F5F3F4F2931A9
:10462000310599F766CF87EC61E070E00E94CD100C
:1046300081E00E94B6100E94AF101092FF030AC0E2
:104640008AEC61E070E00E94CD1080E00E94B6101C
:104650000E94AF10C65ADF4FE6E00C940B30A0E08A
:10466000B0E0E5E3F3E20C94EB2F84E0A82E06E043
:10467000B02E15E0C12E05E315E0B4E6DB2EA2E076
:10468000EA2EF3E0FF2EA1C087E396E00E94A72E5A
:10469000982F8093A00580919F05833021F184306D
:1046A00028F4813099F08230B8F409C0853009F4DB
:1046B00048C0853020F1863009F087C05FC0953B47
:1046C00009F083C081E080939F057FC0923609F096
:1046D0007AC0E0929F0579C090939E0590939D05C6
:1046E000F0929F0572C090939B0510929C0580915B
:1046F0009D05892780939D05A0929F0566C0D92FAF
:10470000C0E020919B0530919C052C2B3D2B3093D4
:104710009C0520939B0580919D05892780939D058D
:10472000C0929F052536310508F44FC08CEC61E03E
:1047300070E00E94CD1081E00E94B6100E94AF1080
:1047400042C02091990530919A05F901EB5CFA4F2E
:10475000908380919D05892780939D052F5F3F4F12
:1047600030939A052093990580919B0590919C0523
:104770002817390750F1B0929F0527C080919D05F9
:10478000891759F46091990570919A0580919E0559
:1047900045E355E00E94B4200DC08BEC62E070E070
:1047A0000E94CD1080919E050E94B6108091000459
:1047B0000E94B610F8018D2D11928A95E9F710929A
:1047C0009A051092990510929F0587E396E00E9442
:1047D0006D2E892B09F058CFCDB7DEB7EAE00C94E7
:1047E000073081E08093FF0308C087E396E00E94D2
:1047F0006D2E892B11F00E942F238091FF038823B7
:10480000A1F70895A0E0B0E0E8E0F4E20C94EE2F08
:104810000E94D9296115710581059105C9F30E948E
:1048200099061092D9031092DA031092DB031092CA
:10483000DC03DD24E090D903F090DA030091DB0380
:104840001091DC03102F0F2DFE2CEE240E949406F5
:104850002FEF30E040E050E00E94C82FE60EF71E38
:10486000081F191FE092D903F092DA030093DB03CB
:104870001093DC03D39444E0D416E1F6CFEDD3E0FB
:1048800000E010E090E1E92E97E2F92E4EC00F5FB4
:1048900019F40E9479084DC00E94940622E330E08A
:1048A00040E050E00E94C82F6F5FEFEDF3E090E032
:1048B00004C08191861759F39F5F9117D0F38091BF
:1048C000DE0390E08E9D90018F9D300D9E9D300DFA
:1048D0001124862F90E0AC01249FC001259F900DEC
:1048E000349F900D1124AA2797FDA095BA2F2091EF
:1048F000D5033091D6034091D7035091D803820F4E
:10490000931FA41FB51F20919D0330919E034091DA
:104910009F035091A003281739074A075B0708F443
:10492000B6CF69931F5F183121F08881882309F081
:10493000AECFCDB7DEB7E7E00C940A301F931091ED
:1049400001041F3F09F0F1C0893409F467C08A34BB
:1049500028F5883309F479C0893368F4803309F481
:1049600086C0813308F06FC08B3109F44DC08132AD
:1049700009F0D5C03DC0813409F49AC0823438F4BE
:10498000893309F472C0803409F0C9C031C082345F
:1049900009F4A1C0863409F0C2C052C0823609F4BD
:1049A0009AC0833690F4883579F1893538F48235A8
:1049B00009F43FC0833509F0B2C01FC08A3509F43D
:1049C000A9C0813609F0ABC073C0823791F183373B
:1049D00030F48636A9F1893609F0A1C01FC08837A6
:1049E00099F08A3709F496C0833709F098C005C05A
:1049F00087E396E069E471E019C00E94B41687E38A
:104A000096E063ED71E006C00E94BD1687E396E074
:104A10006DEE71E00E94282D8EEF7FC00E94790814
:104A20000E94BE0887E396E06CE072E00E94282DA9
:104A300076C00E94022487E396E065E272E0F6CF3A
:104A40000E9465176CC0805368C087E396E06CEEE7
:104A500071E00E94B22B9091F803892F885F8871D2
:104A6000977E892B8093F80320C089E056C087E3A6
:104A700096E069ED71E00E94B22B8091A1039091C4
:104A8000A203A091A303B091A40320E130E040E091
:104A900050E082279327A427B5278093A103909302
:104AA000A203A093A303B093A4031093010437C0FF
:104AB00087E396E063EC71E00E94B22B8091A10342
:104AC0009091A203A091A303B091A40320E430E04D
:104AD00040E050E012C087E396E062EB71E00E9494
:104AE000B22B8091A1039091A203A091A303B09156
:104AF000A40320E230E040E050E082279327A4277F
:104B0000B5278093A1039093A203A093A303B0932E
:104B1000A40302C00E94F11D8FEF809301048091D5
:104B200001048E3F09F4DDC0D4C00E94FC16882326
:104B300009F4D7C080916704882321F48FEF809314
:104B40000104C7C082E094E060E070E040E050E023
:104B50000E94A2069B01AC0180910104992787FD68
:104B60009095A92FB92FFC013197E930F10508F094
:104B70008CC0E753FF4F0C941A30DA01C901815CF5
:104B80009D49A845B5438F5F9945A246B24008F0BC
:104B90007CC02093D5033093D6034093D703509322
:104BA000D8039AC02093D9033093DA034093DB03F0
:104BB0005093DC0381E0809368048EC02830310577
:104BC0004105510508F061C02093DD0385C0DA017D
:104BD000C9010197A109B1090A97A105B10508F01A
:104BE00054C02093DE0378C082E094E06DE371E06E
:104BF0000E94BE0710E00EC0183130F4E12FF0E043
:104C0000E053FC4F87871F5F80E090E06DE371E029
:104C10000E94BE07009759F00E94A007009761F715
:104C200006C0E12FF0E0E053FC4F17861F5F1831FC
:104C3000C0F352C0253031054105510530F52093B0
:104C4000F7034AC0DA01C9010197A109B109069722
:104C5000A105B105D0F48091F803887F822B809361
:104C6000F8033AC0DA01C9010197A109B1098050DE
:104C7000924CA140B04048F42093D1033093D2032A
:104C80004093D3035093D40327C087E396E068EAA8
:104C900071E00E94282D13C08091D9039091DA030E
:104CA000A091DB03B091DC030196A11DB11D80939F
:104CB000D9039093DA03A093DB03B093DC030E9443
:104CC000F2168FEF8093010487E396E06AE00E947A
:104CD000C62B0E94351E05C0809168048823E1F22E
:104CE000EECF1F9108958FEF809301041092680416
:104CF0000E94351E0CC087E396E00E946D2E892B22
:104D000031F087E396E00E94A72E0E949E248091B6
:104D100001048E3F81F76AE070E080E090E00E943D
:104D2000FF2904C087E396E00E94A72E87E396E060
:104D30000E946D2E892BB1F70895AAE2B0E0E3EA54
:104D4000F6E20C94E82F0E94CB297B018C0181E0D4
:104D50000E94661104C087E396E00E94A72E87E3B5
:104D600096E00E946D2E892BB1F75E98DD24D394D6
:104D700052E6752E42E0842E912C8C0E9D1E5E0113
:104D80000894A11CB11C33E0C32E0E94CB2920E063
:104D900030E06E197F09800B910B693C710581052C
:104DA000910510F021E030E08D2D90E0282339238B
:104DB000232B99F10E94CB297B018C015D9A80ED18
:104DC00097E00E940C087982D401E0EDF3E089E2DB
:104DD00001900D928150E1F7C5016AE20E94150F22
:104DE0005D9880E090E00E940C08C0929A030E94B7
:104DF000CC0B62E370E080E090E00E94FF2980919C
:104E00009A03843051F4C0929A038FE70E94C20A39
:104E10000E94D60A823409F4DD248EE00E94FD2A25
:104E2000892B49F5DD24D39426C05E9A5D9A87E3E9
:104E300096E00E94A72E8D30910569F08E30910585
:104E40001CF40A97B1F407C08332910569F08234EB
:104E5000910579F40CC087E396E064EA71E00E9462
:104E6000B22B0E94732605C00E94C81E02C00E9479
:104E7000F1235E985D9887E396E00E946D2E892B62
:104E800009F483CFD2CF8F929F92AF92BF92CF92ED
:104E9000DF92EF92FF920F931F938EE00E94FD2A04
:104EA000892B09F083C068EC70E080E090E00E94FC
:104EB000FF2980E090E00E940C080E94CB295B0152
:104EC0006C0160ECE62E62E1F62E012D112DEA0C4C
:104ED000FB1C0C1D1D1D06C08EE00E94FD2A892BA7
:104EE00009F062C00E94CB296E157F0580079107EB
:104EF00098F38EE00E94FD2A892B09F055C080EDC1
:104F000097E00E940C080E94CB297B018C01992418
:104F10009394882488E496E2A0E0B0E0A80EB91E3D
:104F2000CA1EDB1E29C0AE14BF04C006D10638F469
:104F300080ED97E00E940C08882483941DC00E9495
:104F4000CB296E197F09800B910B693C7105810596
:104F5000910590F00E94CB297B018C0180E0992083
:104F600009F481E0982E882319F480E090E002C0D3
:104F700080ED97E00E940C088EE00E94FD2A892BAC
:104F800091F280E090E00E940C08882049F0809126
:104F90009B038F5F83700E94E2160E94BD1606C0BD
:104FA0000E9402240E94B4160E949D261F910F9118
:104FB000FF90EF90DF90CF90BF90AF909F908F9039
:104FC000089580E06DEF77E042E050E00E9406290E
:104FD0000895EF92FF920F931F9380E00E9445087F
:104FE0000E940B1189E061E00E945E2A89E060E086
:104FF0000E94CA2A86E061E00E945E2A85E061E0A4
:105000000E945E2A8EE060E00E945E2A88E060E0F6
:105010000E945E2A88E061E00E94CA2A81E161E084
:105020000E945E2A81E160E00E94CA2A0E9420114B
:1050300087E396E040E052EC61E070E00E94E62DEC
:105040000E94D5160E94BD160E94AC0C8FEF809373
:10505000BE040E94E12778940E94CB297B018C0139
:105060008091BE048F3F09F0C7C00E94CB296E1902
:105070007F09800B910B605D77408040904008F085
:10508000BBC0EECF87E396E00E94A72E87E396E0B1
:105090000E946D2E892BB1F787E396E062E472E0FF
:1050A0000E94252D80E793E00E946C1A87E396E02A
:1050B00069E572E00E94252D87E396E064E070E0E8
:1050C0004AE050E00E94112D62E370E080E090E041
:1050D0000E94FF2987E396E00E946D2E04970CF151
:1050E00087E396E00E94A72E82349105D1F487E3EE
:1050F00096E00E94A72E8E34910599F487E396E0FE
:105100000E94A72E8434910561F487E396E00E9403
:10511000A72E819731F480E090E00E940C080E9455
:105120009D264091D1035091D2036091D303709199
:10513000D403DB01CA010197A109B1090497A105B4
:10514000B10568F44093BF04433029F040E052ECCD
:1051500061E070E004C040EA56E861E070E087E397
:1051600096E00E94E62D0E9443275E9880E090E042
:105170000E940C080E94AC0C80E00E946611809195
:10518000A4040E94F70A0E94CC0B109229051092E9
:105190002A0510922B0510E015C062E370E080E054
:1051A00090E00E94FF2980ED97E00E940C0862E3E6
:1051B00070E080E090E00E94FF2980E090E00E9493
:1051C0000C081F5F80919B03811738F78091F803CB
:1051D00090E084FF09C020E088719070489709F43E
:1051E00021E0822F0E942F118FE00E9445081F911D
:1051F0000F91FF90EF90089580ED97E00E940C08CA
:105200008EE061E00E94CA2A5E9A40CF823000F5AB
:10521000E82FF0E0EE0FFF1FEE55FA4F7183608329
:10522000882319F08130A1F408C0809169008C7F37
:10523000842B80936900E89A089580916900440F57
:10524000551F440F551F837F842B80936900E99A73
:1052500008951F920F920FB60F9211242F933F9330
:105260004F935F936F937F938F939F93AF93BF936E
:10527000EF93FF938091A2059091A305892B29F0CC
:10528000E091A205F091A3050995FF91EF91BF91DF
:10529000AF919F918F917F916F915F914F913F91CE
:1052A0002F910F900FBE0F901F9018951F920F9285
:1052B0000FB60F9211242F933F934F935F936F93E9
:1052C0007F938F939F93AF93BF93EF93FF938091BF
:1052D000A4059091A505892B29F0E091A405F091F2
:1052E000A5050995FF91EF91BF91AF919F918F9186
:1052F0007F916F915F914F913F912F910F900FBED2
:105300000F901F9018951F920F920FB60F921124B5
:105310002F933F938F939F93AF93BF938091AA0551
:105320009091AB05A091AC05B091AD053091AE0563
:105330000196A11DB11D232F2D5F2D3720F02D5774
:105340000196A11DB11D2093AE058093AA059093EF
:10535000AB05A093AC05B093AD058091A6059091E7
:10536000A705A091A805B091A9050196A11DB11DA1
:105370008093A6059093A705A093A805B093A905CF
:10538000BF91AF919F918F913F912F910F900FBE41
:105390000F901F9018958FB7F8942091AA0530911F
:1053A000AB054091AC055091AD058FBFB901CA0165
:1053B00008959FB7F8942091A6053091A7054091D4
:1053C000A8055091A90586B5A89B06C08F3F21F07E
:1053D0002F5F3F4F4F4F5F4F9FBF542F432F322FB1
:1053E0002227280F311D411D511D82E0220F331F3E
:1053F000441F551F8A95D1F7B901CA010895EF924C
:10540000FF920F931F93CF93DF937B018C010E9438
:10541000D929EB010EC00E94D9296C1B7D0B685E57
:105420007340C8F30894E108F10801091109C85153
:10543000DC4FE114F1040105110569F7CDB7DEB7C2
:10544000E6E00C940B30789484B5826084BD84B51A
:10545000816084BD85B5826085BD85B5816085BD6F
:10546000EEE6F0E0808181608083E1E8F0E0108288
:10547000808182608083808181608083E0E8F0E0C9
:10548000808181608083E1EBF0E0808184608083B3
:10549000E0EBF0E0808181608083EAE7F0E08081EA
:1054A000846080838081826080838081816080834A
:1054B0008081806880831092C1000895CF93DF932C
:1054C000482F50E0CA018D5F934FFC013491415148
:1054D000544FFA018491882369F190E0880F991F55
:1054E000FC01EF52F44FA591B491FC01E552F44F49
:1054F000C591D491662351F42FB7F8948C91932FD2
:10550000909589238C93888189230BC0623061F444
:105510002FB7F8948C91932F909589238C93888141
:10552000832B88832FBF06C09FB7F8948C91832B61
:105530008C939FBFDF91CF910895833071F08430B9
:1055400028F48130A1F0823021F514C08630B1F00A
:105550008730D1F08430E9F404C0809180008F77E7
:1055600003C0809180008F7D80938000089584B572
:105570008F7702C084B58F7D84BD08958091B0007F
:105580008F778093B00008958091B0008F7D8093D5
:10559000B0000895FF920F931F93F62E482F50E00E
:1055A000CA01895E934FFC012491CA018D5F934F1C
:1055B000FC0114914151544FFA0104910023C9F0A8
:1055C000222319F0822F0E949D2AE02FF0E0EE0F97
:1055D000FF1FE552F44FA591B4919FB7F894FF20B7
:1055E00021F48C911095812302C08C91812B8C9396
:1055F0009FBF1F910F91FF9008950F931F93482F06
:1056000050E0CA01895E934FFC012491CA018D5F6D
:10561000934FFC0104914151544FFA01149111230D
:1056200019F420E030E015C0222319F0822F0E94E7
:105630009D2A812F90E0880F991F8B51944FFC0178
:10564000A591B4918C9120E030E0802311F021E00D
:1056500030E0C9011F910F910895982F8E3008F006
:105660009E509770809148038295880F880F807CA8
:10567000892B80937C0080917A00806480937A00EB
:1056800080917A0086FDFCCF2091780040917900CE
:10569000942F80E030E0282B392BC9010895A0E039
:1056A000B0E0E5E5FBE20C94ED2F7C016B018A0193
:1056B000C0E0D0E00FC0D6016D916D01D701ED9132
:1056C000FC910190F081E02DC7010995C80FD91F09
:1056D000015010400115110571F7CE01CDB7DEB7AD
:1056E000E8E00C940930EF92FF920F931F93CF9351
:1056F000DF937C018B01C0E0D0E0F8010F5F1F4F0A
:105700006491662359F0D701ED91FC910190F081ED
:10571000E02DC7010995C80FD91FEFCFCE01CDB736
:10572000DEB7E6E00C940B30DC01ED91FC910190CA
:10573000F081E02D09950895EF92FF920F931F934A
:105740008C016DE00E94942B7C01C8016AE00E94EC
:10575000942B9C012E0D3F1DC9011F910F91FF90AD
:10576000EF900895EF92FF920F931F937C010E9498
:10577000732B8C01C7010E949C2B9C01200F311FB1
:10578000C9011F910F91FF90EF900895EF92FF9242
:105790000F931F937C010E94942B8C01C7010E94E0
:1057A0009C2B9C01200F311FC9011F910F91FF906D
:1057B000EF900895CF93DF93EC016115710519F413
:1057C00020E030E00FC0DB010D900020E9F71197D9
:1057D000A61BB70BE881F9810280F381E02DAD01B2
:1057E00009959C01C901DF91CF9108954F925F9275
:1057F0007F928F929F92AF92BF92CF92DF92EF9261
:10580000FF920F931F93DF93CF93CDB7DEB7A1978E
:105810000FB6F894DEBF0FBECDBF2C01742ECB01A6
:10582000223008F42AE019A231E2C32ED12CCC0E8A
:10583000DD1E822E9924AA24BB24672D752FA50175
:1058400094010E94A62F79018A01C801B701A50120
:1058500094010E94742F472D461B0894C108D1085B
:105860004A3010F4405D01C0495CF6014083E11408
:10587000F1040105110521F07E2C5F2DC801DDCF5B
:10588000C201B6010E94DA2BA1960FB6F894DEBFD2
:105890000FBECDBFCF91DF911F910F91FF90EF9081
:1058A000DF90CF90BF90AF909F908F907F905F9050
:1058B0004F900895DC012115310541F4ED91FC91E3
:1058C0000190F081E02D642F099508950E94F62B38
:1058D0000895EF92FF920F931F937C010E945A2C20
:1058E0008C01C7010E949C2B9C01200F311FC90114
:1058F0001F910F91FF90EF900895EF92FF920F93F9
:105900001F939A017B0100E010E0B801A7010E94FB
:105910005A2C1F910F91FF90EF900895EF92FF92F4
:105920000F931F937C010E947D2C8C01C7010E9464
:105930009C2B9C01200F311FC9011F910F91FF90DB
:10594000EF900895EF92FF920F931F939A01E62E26
:10595000FF2400E010E0B801A7010E945A2C1F911B
:105960000F91FF90EF900895EF92FF920F931F9386
:105970007C010E94A22C8C01C7010E949C2B9C01DF
:10598000200F311FC9011F910F91FF90EF900895D3
:10599000A0E0B0E0EEECFCE20C94ED2FEC016A012B
:1059A0007B012115310541F4E881F9810190F081F5
:1059B000E02D642F09951BC02A303105B1F477FF23
:1059C00013C06DE20E94942B8C0144275527BA0125
:1059D0004C195D096E097F09CE012AE00E94F62B61
:1059E0009C01200F311F04C02AE00E94F62B9C016D
:1059F000C901CDB7DEB7E8E00C940930EF92FF9211
:105A00000F931F937B019A010027F7FC0095102F3D
:105A1000B801A7010E94C82C1F910F91FF90EF9031
:105A20000895EF92FF920F931F937C010E94FE2C2A
:105A30008C01C7010E949C2B9C01200F311FC901C2
:105A40001F910F91FF90EF9008950E94DA2B089517
:105A5000EF92FF920F931F937C010E94252D8C01E2
:105A6000C7010E949C2B9C01200F311FC9011F916F
:105A70000F91FF90EF90089508951F920F920FB627
:105A80000F9211242F933F934F938F939F93EF93F4
:105A9000FF938091C00082FD1DC04091C6002091FF
:105AA000EF053091F0052F5F3F4F2F7330708091DD
:105AB000F1059091F2052817390771F0E091EF0593
:105AC000F091F005E155FA4F40833093F0052093B3
:105AD000EF0502C08091C600FF91EF919F918F91D9
:105AE0004F913F912F910F900FBE0F901F901895DF
:105AF0001F920F920FB60F9211242F933F938F9303
:105B00009F93EF93FF932091330630913406809159
:105B10003506909136062817390731F48091C10077
:105B20008F7D8093C10014C0E0913506F091360658
:105B3000ED50FA4F208180913506909136060196FE
:105B40008F73907090933606809335062093C6002D
:105B5000FF91EF919F918F913F912F910F900FBEE9
:105B60000F901F901895A0E0B0E0E9EBFDE20C94D7
:105B7000E92FFC011382128288EE93E0A0E0B0E0EE
:105B800084839583A683B7838BE893E09183808396
:105B90007587648757874687318B208B138B028BE1
:105BA000F58AE48AD78AC68AB18EA08E938E828EB9
:105BB0008F85848F8889858F8989868F8A89878F49
:105BC0008B8980A32096ECE00C940530AF92BF92B5
:105BD000DF92EF92FF920F931F93CF93DF93EC012D
:105BE0007A018B01DD24403081EE580780E06807A0
:105BF00080E0780711F0DD24D39491E0A92EB12C38
:105C0000EC89FD89DD2069F0C50108A002C0880F7C
:105C1000991F0A94E2F7808360E079E08DE390E0D9
:105C200005C0108260E874E88EE190E0A801970159
:105C30000E94A62F21503040404050405695479535
:105C40003795279580E12030380720F0DD2011F0CE
:105C5000DD24D6CFE889F9893083EA89FB8920835E
:105C600019A2EE89FF89408121E030E0C9010C8C46
:105C700002C0880F991F0A94E2F7482B4083EE89EF
:105C8000FF894081C9010D8C02C0880F991F0A94B9
:105C9000E2F7482B4083EE89FF894081C9010E8CD1
:105CA00002C0880F991F0A94E2F7482B4083EE89BF
:105CB000FF8980810F8C02C0220F331F0A94E2F704
:105CC000209528232083DF91CF911F910F91FF9082
:105CD000EF90DF90BF90AF900895DC011C96ED919E
:105CE000FC911D97E05CFF4F219131918081918162
:105CF000281B390B2F733070C901089587E396E094
:105D00000E946D2E892B11F00E943C2D0895DC011C
:105D10001C96ED91FC911D97E05CFF4F2081318135
:105D2000E054F040DF01AE5BBF4F8D919C91119725
:105D30002817390719F42FEF3FEF07C08D919C9179
:105D4000E80FF91F8081282F30E0C9010895DC0198
:105D50001C96ED91FC911D97E05CFF4F20813181F5
:105D6000E054F040DF01AE5BBF4F8D919C911197E5
:105D70002817390719F42FEF3FEF10C08D919C9130
:105D80001197E80FF91F20818D919C911197019631
:105D90008F73907011969C938E9330E0C901089593
:105DA000DC0191968C919197882339F05496ED916E
:105DB000FC915597808186FFF9CF91961C920895AA
:105DC000CF93DF93EC01EE85FF85E05CFF4F2081F0
:105DD0003181E054F0402F5F3F4F2F733070DF016F
:105DE000AE5BBF4F8D919C91119728173907D1F366
:105DF000E05CFF4F80819181E054F040E80FF91F93
:105E00006083EE85FF85E05CFF4F31832083EE8960
:105E1000FF89208181E090E00F8C02C0880F991FDC
:105E20000A94E2F7282B208381E089A3EC89FD897D
:105E300080818064808381E090E0DF91CF9108953C
:105E40008F929F92AF92BF92CF92DF92EF92FF928A
:105E50000F931F9300D000D00F92EDB7FEB731968D
:105E600084E0ADB7BEB711968C9383E0818387E061
:105E7000828385E0838381E0848387E396E06FEA11
:105E800075E043EF55E025EC30E004EC10E0B0ECB9
:105E9000EB2EF12CA1ECCA2ED12CF2ECAF2EB12CB2
:105EA000E6EC8E2E912C0E94B32D0F900F900F9048
:105EB0000F900F901F910F91FF90EF90DF90CF9078
:105EC000BF90AF909F908F900895CF93DF930E94E3
:105ED000232A0E94E927CEE7DEE20E94591220978A
:105EE000E1F30E947E2EF9CF629FD001739FF001F3
:105EF000829FE00DF11D649FE00DF11D929FF00D5A
:105F0000839FF00D749FF00D659FF00D9927729F90
:105F1000B00DE11DF91F639FB00DE11DF91FBD011B
:105F2000CF011124089597FB092E07260AD077FD8B
:105F300004D086D006D000201AF4709561957F4F6A
:105F40000895F6F7909581959F4F0895A1E21A2E36
:105F5000AA1BBB1BFD010DC0AA1FBB1FEE1FFF1F0D
:105F6000A217B307E407F50720F0A21BB30BE40B5D
:105F7000F50B661F771F881F991F1A9469F76095A4
:105F80007095809590959B01AC01BD01CF0108955E
:105F900097FB092E05260ED057FD04D0D7DF0AD077
:105FA000001C38F450954095309521953F4F4F4F48
:105FB0005F4F0895F6F790958095709561957F4FA6
:105FC0008F4F9F4F08952F923F924F925F926F9203
:105FD0007F928F929F92AF92BF92CF92DF92EF9279
:105FE000FF920F931F93CF93DF93CDB7DEB7CA1BFA
:105FF000DB0B0FB6F894DEBF0FBECDBF09942A8825
:10600000398848885F846E847D848C849B84AA84CC
:10601000B984C884DF80EE80FD800C811B81AA8159
:10602000B981CE0FD11D0FB6F894DEBF0FBECDBF24
:10603000ED010895EE0FFF1F0590F491E02D0994F6
:10604000AA1BBB1B51E107C0AA1FBB1FA617B7079E
:1060500010F0A61BB70B881F991F5A95A9F78095BA
:106060009095BC01CD010895911106C0803219F0C0
:1060700089508550D0F70895992788270895F89476
:02608000FFCF50
:106082004E6F005965730054582074696D656F75C1
:106092007421006D6F64756C65206C6F636B656451
:1060A2003F00486F70206368616E6E656C2000204F
:1060B20040200053004E2F4100386368002C002C12
:1060C200205B005D20280029004E4F5420454E41A0
:1060D200424C45440053656E64696E672073657473
:1060E20074696E677320746F2052580A0052657388
:1060F200657474696E672073657474696E67732062
:106102006F6E2052580A0041626F72746564206596
:10611200646974730A00696E76616C6964207365E0
:106122006C656374696F6E000D0A496E76616C6905
:106132006420696E707574202D20646973636172C6
:106142006465642107007363616E6E6572206D6F12
:1061520064650053657474696E6773207361766554
:106162006420746F20454550524F4D0A00526576A7
:1061720065727465642073657474696E67732066F2
:10618200726F6D20454550524F4D0A004C6F61644D
:10619200656420666163746F7279206465666175F7
:1061A2006C74730A004B657920616E6420636861C8
:1061B2006E6E656C732072616E646F6D697A656470
:1061C2000A004F70656E4C52536E6720545820730C
:1061D20074617274696E672000206F6E20485720C8
:1061E2000050504D00525353490053444100534311
:1061F2004C00525844005458440041494E004C420D
:106202004545500053504B54524D00534255530094
:1062120053554D44004C4C494E440000342B34003D
:106222003800382B340031320031322B3400313611
:106232000001000000C01200001A400AA1204EA571
:10624200001B1E27522C23308025000005400AA186
:10625200204EA50020244EA52C2330004B00000622
:10626200400AD0009D49007B289D492C233000E143
:10627200000005400A4501D7DC03B81E0EBF00230B
:106282002E48E801008A400A6001555502AD1E20E1
:10629200000023C88025000005400AA1204EA50069
:1062A20020244EA52C23300002000200020002002E
:1062B20002000200020002000200020002000200CC
:1062C20002000200020002FF01610265026A026E20
:1062D20002720276027A027E0284028B0290029598
:1062E200029B029B029B029B0235019C02A002A21E
:1062F20002A602A902AE02350100070B0C1011150D
:1063020000160A1322312900000000E02E4F2B6DE7
:086312002EA72E872ED02E00CD
:107E00000F92CDB7DEB7112484B714BE81FFF1D035
:107E100082E08093C00088E18093C10086E0809377
:107E2000C20080E18093C4008EE0CDD088249924E4
:107E3000CC24C394F5E0DF2EE1E1EE2E73E0F72EC3
:107E4000B6D0082F813479F4B2D08983C2D0898129
:107E5000823811F481E005C0813811F485E001C059
:107E600083E09ED09AC0823411F484E103C085344B
:107E700019F485E0B6D091C0853561F498D0082F0B
:107E800010E095D090E0982E8824802A912A880CC2
:107E9000991C82C0863521F484E0A3D080E0E1CF34
:107EA000843609F04CC083D082D0A82E80D0B82E62
:107EB00000E011E07CD0F80181938F01AE16D1F77C
:107EC00088D0FB2DF53489F4E0E0F1E00BC0F9999E
:107ED000FECF92BC81BC0894811C911C819180BD15
:107EE000FA9AF99AEA1598F358C08B2D863409F05E
:107EF00054C0F401F7BEE89507B600FCFDCFF401CD
:107F0000A0E0B1E02C9130E011968C91119790E0B7
:107F1000982F8827822B932B12960C01C7BEE895C9
:107F20001124329681E0A038B80761F7F401D7BE7A
:107F3000E89507B600FCFDCFE7BEE8952EC0843774
:107F4000F1F435D034D0182F32D0B82E42D0FB2DDA
:107F5000F63421F4F40105914F010CC0FB2DF534EA
:107F600049F4F999FECF92BC81BC0894811C911C04
:107F7000F89A00B5802F14D0115049F70EC08537FC
:107F800039F427D08EE10CD085E90AD08FE069CF93
:107F9000813511F488E017D01CD080E101D050CF9A
:107FA0009091C00095FFFCCF8093C600089580910A
:107FB000C00087FFFCCF8091C00084FD01C0A89560
:107FC0008091C6000895E0E6F0E098E19083808318
:107FD0000895EDDF803219F088E0F5DFFFCF84E10E
:107FE000DFCF1F93182FE3DF1150E9F7F2DF1F9166
:0E7FF0000895282E80E0E7DFEE27FF27099492
:027FFE0001057B
:0400000300007E007B
:00000001FF
